:103800000C94241C0C943F1C0C943F1C0C943F1CE7
:103810000C943F1C0C943F1C0C943F1C0C943F1CBC
:103820000C943F1C0C943F1C0C943F1C0C943F1CAC
:103830000C943F1C0C943F1C0C943F1C0C943F1C9C
:103840000C943F1C0C943F1C11241FBECFE5D4E008
:10385000DEBFCDBF10E0A0E6B0E0EEE4FFE302C0C3
:1038600005900D92A036B107D9F711E0A0E6B0E0BF
:1038700001C01D92A43AB107E1F70C946C1F0C949F
:10388000001C0F93EF93FF933ED0FC01062F35D021
:10389000FF91EF910F9108950F930F921F92EF9365
:1038A000FF9331D0FC010B0101E027D0FF91EF9194
:1038B0001F900F900F9108950F930F92EF93FF9326
:1038C00022D0FC0160FD67BFC895802DE395C895A7
:1038D000902DFF91EF910F900F9108950F930F92FC
:1038E00012D0082E09E009D00F900F9108950F9380
:1038F0000AD001E102D00F910895E199FECF07BFF0
:10390000E895FFFF000007B700FDFDCF089583E0B5
:1039100089B9549A539A08958CB19927089540E033
:1039200050E04817590750F427EE33E000002150CB
:10393000304037FFFBCF4F5F5F4FF3CF08958BB120
:1039400099278078907008955498539808950E940C
:10395000A41C0C94000008958CB95E9BFECF5E9A67
:1039600008950E949F1C8823E1F30E948C1C8032E2
:1039700019F481E090E0089585E10E94AC1C80E09C
:1039800090E008950895EF92FF920F931F93CF93C5
:10399000DF937B01C0E0D0E0C617D70770F48C013D
:1039A0000E949F1C8823E1F30E948C1CF8018193E4
:1039B0008F012196CE15DF0598F381E090E0DF912D
:1039C000CF911F910F91FF90EF90089590E0282FD5
:1039D00033272138310589F02238310524F4203885
:1039E000310549F00DC02238310549F0283931053B
:1039F00039F493E005C092E003C091E001C092E188
:103A0000892F9927089540E050E06091A0007091BF
:103A1000A10046175707E8F4E2EAF0E08091A2011E
:103A20008EBB8091A2019091A301292F33272FBB38
:103A300001969093A3018093A20180818DBBE29AAD
:103A4000E19AE199FECF4F5F5F4F319646175707D6
:103A500028F308950F931F93CF93DF9300E010E0B6
:103A60008091A0009091A10008171907D8F4C2EA2C
:103A7000D0E08091A2019091A301880F991F60E08E
:103A8000800F911F0E945C1C8883892F992789834E
:103A90000E5F1F4F22968091A0009091A100081701
:103AA000190738F3DF91CF911F910F9108958091FD
:103AB000A0009091A1000097C1F0E2EAF0E0AC0113
:103AC0008091A2018EBB8091A2019091A301292F28
:103AD00033272FBB01969093A3018093A201E09A14
:103AE0008DB381934150504059F708950F931F9320
:103AF000CF93DF938C016115710541F0EB01F80163
:103B000081918F010E94AC1C2197C9F781E090E060
:103B1000DF91CF911F910F910895EF92FF920F9334
:103B20001F93CF93DF93C0E0D0E08E017E01CFE7FB
:103B3000D0E0F092A301E092A20163E0C8010E94EC
:103B4000411C219780E490E0E80EF91E00581F4FB9
:103B5000D7FFEFCF0E94771CDF91CF911F910F917C
:103B6000FF90EF900895EF92FF920F931F93CF93E2
:103B7000DF9300E010E08091A0009091A100081771
:103B8000190708F047C0EE24FF24E801CD55DF4FA8
:103B9000F801EE55FF4FEE0DFF1D40818881229602
:103BA0009927382F2227240F311D8091A20190914F
:103BB000A301880F991FB9018E0D9F1D0E944C1CF7
:103BC00082E090E0E80EF91E90E8E916F10400F3B7
:103BD0008091A2019091A301880F991F63E0800F4B
:103BE000911F0E94411C8091A2019091A301880F16
:103BF000991F65E0800F911F0E94411C0E94771C55
:103C000000581F4F8091A0009091A100081719073C
:103C100008F4B9CFDF91CF911F910F91FF90EF90F2
:103C20000895CF93C0E069E081E090E00E945C1CC1
:103C300084FF03C08F7E0E946E1C0E949F1C8823FD
:103C4000E1F30E948C1C992782359105DCF48035C4
:103C500091050CF054C08134910509F45AC08234A6
:103C600091053CF48033910509F449C0C19759F19D
:103C70002FC18234910509F45FC08534910509F4A0
:103C80005EC026C18635910509F4EDC087359105E2
:103C90004CF48235910509F461C08535910509F42C
:103CA00065C016C18437910509F4A0C08537910518
:103CB0002CF48436910509F472C00AC18537910548
:103CC00009F4C1C005C10E94B11C882309F4B5CF15
:103CD00084E10E94AC1C81E40E94AC1C86E50E9439
:103CE000AC1C82E50E94AC1C80E20E94AC1C83E507
:103CF0000E94AC1C84E50E94AC1C8BE406C00E94B0
:103D0000B11C882309F499CF84E10E94AC1C80E1A6
:103D1000E0C061E070E080E690E00E94C31C0E9479
:103D2000B11C882309F489CF84E10E94AC1C8091E6
:103D300060000E94E61CE9CF64E170E00AC061E027
:103D400070E080E690E00E94C31C8091600099279B
:103D5000BC0180E690E00E94C31CD1CF0E94B11C40
:103D6000882309F46ACF0E948D1DCECF62E070E0F7
:103D700080E690E00E94C31C0E94B11C882309F4D5
:103D80005CCF20916000809161009927982F88274F
:103D9000820F911D9093A3018093A201B5CF63E0A0
:103DA00070E080E690E00E94C31C20916100809149
:103DB00060009927982F8827820F911D9093A1006A
:103DC0008093A000BC0182EA90E00E94C31C0E9484
:103DD000B11C882309F431CF80916200863419F434
:103DE0000E94B31D91CF0E94031D8ECF63E070E04F
:103DF00080E690E00E94C31C2091610080916000E9
:103E00009927982F8827820F911D9093A100809366
:103E1000A0000E94B11C882309F40FCF809162009A
:103E2000863419F40E942A1D02C00E94571D84E1A5
:103E30000E94AC1C6091A0007091A10082EA90E009
:103E40000E94761D64CF0E94B11C882309F4F5CE30
:103E500084E10E94AC1C8EE10E94AC1C84E90E94AB
:103E6000AC1C82E052CF64E070E080E690E00E94FB
:103E7000C31C0E94B11C882309F4DFCE84E10E9498
:103E8000AC1C80916000803531F480916100882302
:103E900061F4C82F17C0883531F4809161008830F3
:103EA00061F4C3E00FC0803531F480916100883047
:103EB00049F4C2E007C0883529F480916100882365
:103EC00009F4C1E069E08C2F99270E945C1C1DCF8A
:103ED00085E10E94AC1CB1CECFE5D4E0DEBFCDBF02
:103EE000CEE1F8948EEF91E00E949E1F843B59F43E
:103EF0008FEF91E00E949E1F833C29F48DEF91E0AB
:103F00000E949E1F81BF0E94871C0E948C1C84E619
:103F100090E00E948F1C0E949F1C882321F4C150B6
:103F2000C8BBCC23A1F7CC2319F00E94111E02C0FC
:103F30000E94A71C80E090E00C94A61FE199FECFA0
:0E3F40009FBB8EBBE09A99278DB30895FFCFEB
:0400000300003800C1
:00000001FF
